S01900006F70656E626C745F73746D3332683734332E73726563F9
S3150800000000000220F157000841580008415800082E
S3150800001041580008415800084158000800000000EF
S315080000200000000000000000000000004158000821
S31508000030415800080000000041580008790B0008E4
S31508000040415800084158000841580008415800081E
S31508000050415800084158000841580008415800080E
S3150800006041580008415800084158000841580008FE
S3150800007041580008415800084158000841580008EE
S3150800008041580008415800084158000841580008DE
S3150800009041580008415800084158000841580008CE
S315080000A041580008415800084158000841580008BE
S315080000B041580008415800084158000841580008AE
S315080000C0415800084158000841580008415800089E
S315080000D0415800084158000841580008415800088E
S315080000E0415800084158000800000000415800081F
S315080000F0415800084158000841580008415800086E
S31508000100415800084158000841580008415800085D
S31508000110415800084158000841580008415800084D
S31508000120415800084158000841580008415800083D
S31508000130415800084158000841580008415800082D
S3150800014000000000000000000000000000000000A1
S31508000150415800084158000841580008415800080D
S3150800016041580008415800084158000841580008FD
S31508000170415800084158000841580008000000008E
S3150800018041580008415800084158000841580008DD
S3150800019041580008415800084158000841580008CD
S315080001A041580008415800084158000841580008BD
S315080001B041580008415800084158000841580008AD
S315080001C0415800084158000841580008415800089D
S315080001D0415800084158000841580008415800088D
S315080001E0415800084158000841580008415800087D
S315080001F0415800084158000841580008415800086D
S31508000200415800084158000841580008415800085C
S31508000210415800084158000841580008415800084C
S3150800022041580008415800084158000800000000DD
S3150800023041580008415800080000000041580008CD
S31508000240415800084158000841580008415800081C
S31508000250415800084158000841580008415800080C
S3150800026041580008415800084158000841580008FC
S31508000270415800084158000841580008000000008D
S31508000280415800084158000841580008000000007D
S30D080002900000000041580008B7
S3150800029810B5054C237833B9044B13B10448AFF3AA
S315080002A800800123237010BDC40000200000000050
S315080002B82C5D000808B5034B1BB103490348AFF387
S315080002C8008008BD00000000C80000202C5D00085A
S315080002D872B6704762B67047F0B5184D2C6D24F0A3
S315080002E840542C65002401E00134E4B2112C23D8CB
S315080002F8134D15F8146005EB44056F78F51905FBD9
S3150800030800054FF4FA5EBEFBF5FE05FB0EF5B5F5DE
S31508000318FA5FE9D135463D4405FB000E4FF4FA5518
S31508000328B5FBFEF50D80013DADB2B5F5007FDBD214
S3150800033816701F700120F0BD0020F0BD0044025859
S31508000348B85D000870B58AB00022ADF826208DF889
S3150800035825200AAB03F8042D0DF125020DF1260117
S315080003684FF4FA70FFF7B8FF00283CD0204C214B11
S3150800037823600025A560E560012626746574A574C2
S31508000388BDF826306361A6619DF82530E3619DF8BE
S31508000398243023626662A662E66226636563A663FC
S315080003A8E563256404236364A564E36426656365D5
S315080003B8A565E66525666566A366204601F03CFBE5
S315080003C80195029503960723049340F267630593FC
S315080003D80693079501A9204601F078FC204601F006
S315080003E8B8FC0AB070BDB821034800F0A9FDBDE7FE
S315080003F8E000002000A00040905D000810B58AB013
S3150800040840F2E173019300230293039309040491CC
S3150800041805930693079308935223099301230246E3
S3150800042801A90E4801F0AFFC08B10AB010BD0121B8
S315080004380A4801F0DEFC0028F7D100F08DFB00F130
S3150800044832040121054801F0DCFD0028EDD000F052
S3150800045881FE00F081FB8442F3D2E6E7E000002043
S3150800046830B58BB004460D460021104801F0A2FDB0
S3150800047860B90120B0B940F26763009A9A420CD075
S31508000488002080B19DF80E302B700CE023466A4692
S315080004980021064801F0C0FCECE7019B002BF0D1CF
S315080004A80120EEE700200BB030BD00BFE0000020B9
S315080004B808B5FFF70DFF08BD10B500F057FA00B9E3
S315080004C810BD01F047F80028FAD000F0EDFD00F05D
S315080004D81BFB01F093F800F04DFA054B0340054A5B
S315080004E8936000F047FA4468FFF7F4FEA047E7E789
S315080004F880FFFF1F00ED00E070B508E0461C4D1CA4
S315080005080B78037000F026FE304629462246531E0D
S315080005189CB2002AF2D170BD38B50546002401E020
S315080005280134E4B20E2C12D800F014FE04EB44028F
S315080005389300084AD358AB42F2D804EB4402910018
S31508000548044A0A44526813449D42E9D200E0FF244B
S31508000558204638BDDC5D000810B5C1F309031BB990
S3150800056801241CB9204610BD0024FAE703689942FD
S31508000578F8D040F8041B4FF48062FFF7BDFFF1E797
S315080005882DE9F04107460068FFF7C6FFFF2807D0A0
S315080005984FF00108B8F1000F05D14046BDE8F081D3
S315080005A84FF00008F6E701F035FD002605E04FF0A4
S315080005B80008B8F1000F1DD001361F2E1AD83D685D
S315080005C8740125443C44043400F0C4FD22462946F7
S315080005D8012001F0E9FD58B900231F2BE9D8E95C89
S315080005E8C9B2E25CD2B29142E1D10133DBB2F4E797
S315080005F84FF0000801F03CFDCFE7000070B50E4645
S315080006080E4B984208D004460D4B994207D0FFF77F
S31508000618B7FF70B1254604E00A4D2C4601E0074DA0
S315080006282C4625B131462046FFF796FF18B12846CD
S3150800063870BD0025F5E70025F9E700BF8405002009
S3150800064800000208800100202DE9F84306460C46FA
S3150800065817461D46DFF88C8001EA08080368B3F1D7
S31508000668FF3F0AD04FF00109B9F1010F0ED0B9F1D1
S31508000678010F18D04846BDE8F8834146FFF76CFFD6
S3150800068881460028F0D04FF00109EDE73368984510
S31508000698EDD041463046FFF7B1FF06460028E6D1B9
S315080006A84FF00009E3E73368E41A3444043405E0F4
S315080006B817F8013B04F8013B013DDBD000F04AFD81
S315080006C8331DE31AB3F5806FF2D308F58061304617
S315080006D8FFF794FF064608B1041DE9E74FF000093D
S315080006E8C8E700BF00FCFFFF70B586B004460D4694
S315080006F800230093884205D801262EB946B9304604
S3150800070806B070BD0026F8E70E2DF7D90026F5E7DE
S3150800071801F080FCAC4227D800F01CFD154963009F
S3150800072823449A008B188A585B68002B18BFB2F1C5
S31508000738FF3F18D000230193202305930A46630038
S315080007481819810008461144497A02910244137A15
S31508000758039301230493694601A801F0EFFD30B914
S315080007680134E4B2D6E7002601F082FCC7E7002682
S31508000778FAE700BFDC5D00084FF0FF33024A136052
S31508000788024A1360704700BF8001002084050020D4
S31508000798F8B505460E4617464A1E184B1B1A9A42BE
S315080007A806D80124012C05D0012C12D02046F8BD04
S315080007B80024F7E72846FFF7AFFEFF2807D0701989
S315080007C80138FFF7A9FEFF28EED10024ECE700243C
S315080007D8EAE70B4B2B400B4A934207D033463A4677
S315080007E829460948FFF730FF0446DFE733463A4605
S315080007F829460648FFF728FF0446D7E7FFFF1F08DC
S3150800080800FCFFFF00000208800100208405002084
S31508000818F8B506460D464A1E114B1B1A9A4208D8C1
S315080008280124012C07D0FF210F46012C12D020469F
S31508000838F8BD0024F5E73046FFF76EFE0746A81907
S315080008480138FFF769FE0146FF2818BFFF2FECD1CC
S315080008580024EAE73846FFF747FF0446E7E700BFFC
S31508000868FFFF1F08104B1B68B3F1FF3F1AD000B5EE
S3150800087883B00D4A536891680B44D1680B441169D3
S315080008880B4451690B4491690B44D26913445B4282
S3150800089802AA42F8043D04210448FFF779FF03B089
S315080008A85DF804FB012070478405002098020208B9
S315080008B80D4B1B680D4A126813440D4A12681344F7
S315080008C80C4A126813440C4A126813440B4A1268F5
S315080008D813440B4A126813440A4A1268D34201D0D1
S315080008E8002070470120704700000208040002082B
S315080008F8080002080C000208100002081400020882
S31508000908180002089802020810B50E4B1B68B3F1C6
S31508000918FF3F06D00B48FFF733FE044610B1012403
S3150800092800E00124012C01D0204610BD064B1B68A7
S31508000938B3F1FF3FF8D00448FFF722FE0028F3D1A9
S315080009480446F1E784050020800100200048704726
S315080009580000020808B5FFF70FFF08BD08B5FFF73E
S3150800096817FF08BD08B5FFF753FF08BD08B5FFF719
S315080009789FFF08BD08B5FFF7E9FF08BD08B5FFF7EB
S3150800098871FF034608B9184608BDFFF7BDFF0346B9
S31508000998F9E70000074BDB6913F0200F06D001239F
S315080009A833B1044B5B6A0370012070470023F7E7ED
S315080009B8002070470048004010B50B4B986200F0BD
S315080009C8CBF800F10A0407E0012363B900F0C2FB7B
S315080009D800F0C2F8844206D3034BDB6913F0800F94
S315080009E8F2D10023F1E710BD0048004010B588B0E1
S315080009F8002300934FF461420192029303930493F0
S31508000A080C22059206930793054C6946204603F07F
S31508000A188BF9236843F00103236008B010BD00BFB3
S31508000A280048004070B506460D46402904D82846B1
S31508000A38FFF7C2FF00240BE08221074800F080FA7E
S31508000A48F5E700F087FB305DFFF7B6FF0134A4B27F
S31508000A58ABB29C42F5D370BD905E000870B5254BC5
S31508000A681C78BCB92448FFF795FF012801D0204611
S31508000A7870BD214B1B78013BDBB23F2BF7D800F042
S31508000A886BF81E4B186000221D4B1A700122194B71
S31508000A981A70ECE706460D46194B1B7801331648BB
S31508000AA81844FFF777FF044601280AD000F054F8DF
S31508000AB8124B1B686433984219D900240D4B1C70D5
S31508000AC8D5E70F4B1A780132D2B21A700A4B1B783F
S31508000AD89A4201D00024CAE70A493046FFF70CFDB6
S31508000AE80022044B1A70064B1B782B70BFE70024AC
S31508000AF8BDE700BFC909002088090020CC090020E5
S31508000B08CA090020890900200022014B1A6070478B
S31508000B1810E000E008B5FFF7F7FF054B054A5A60ED
S31508000B2800229A6005211960034B1A6008BD00BFA8
S31508000B3810E000E0FF520700D0090020044B1B68AC
S31508000B4813F4803F03D0034A1368013313607047D0
S31508000B5810E000E0D009002008B5FFF7EFFF014BC9
S31508000B68186808BDD009002008B5FFF7F5FF08BDC5
S31508000B7870470000094B03F11801002232B19A7434
S31508000B8800225A61054A064B1A6070479A745961D9
S31508000B98183318310132D2B2F0E700BF140A002020
S31508000BA8440A00200A4B1B6883B110B45C69084ADA
S31508000BB8146019749860D86000225A74186001394C
S31508000BC808445860987C5DF8044B7047FF207047C6
S31508000BD8440A002038B504460D46012804D94FF4BE
S31508000BE8E171124800F0ACF962002244D100104BBA
S31508000BF80B445A7C1B7C9A4213D00D4B0B44DA687B
S31508000C0815705A7C01325A74DA680132DA605B6800
S31508000C189A4208D9064A084651580244D160012022
S31508000C2838BD002038BD012038BD00BFBC5E0008AD
S31508000C38140A002008B50146024B1878FFF7CAFFC0
S31508000C4808BD00BF480A002038B504460D460128E5
S31508000C5804D94FF4F271134800F072F904EB44030F
S31508000C68DA00114B13445B7CBBB162002244D10005
S31508000C780D4B0B449A6812782A705A7C013A5A74B2
S31508000C889A6801329A605B689A4208D9064A084601
S31508000C98515802449160012038BD002038BD012012
S31508000CA838BD00BFBC5E0008140A002008B5014616
S31508000CB8024B1878FFF7C8FF08BD00BF8C0A00204A
S31508000CC810B50446012804D94FF40171044800F008
S31508000CD837F904EB4404E200024B1344587C10BD70
S31508000CE8BC5E0008140A002038B5FFF743FF1B4C02
S31508000CF84021601CFFF756FF2070194D4021681CDB
S31508000D08FFF750FF28702378FF2B1DD0FF281BD02C
S31508000D18144C00221449204603F02AFE134920469B
S31508000D2803F04FFE012000F030FC204603F050FE89
S31508000D3802F0E2F9D4F8C00202F00AF800F02CF939
S31508000D48B0F5FA6F05D338BD8521094800F0F8F8DB
S31508000D58DEE74FF4FA6000F019F9F4E7480A0020CC
S31508000D688C0A0020D00A00207400002010000020F9
S31508000D78BC5E000810B5064CD4F8C00202F006F8A6
S31508000D88204603F00CFE002000F0FFFB10BD00BF54
S31508000D98D00A002070B506460D463F290AD82846C7
S31508000DA8FFF748FF012803D0BF210E4800F0C8F80E
S31508000DB8002406E0BB210B4800F0C2F8EFE701342F
S31508000DC8A4B2ABB29C420BD200F0C4F9305DFFF76F
S31508000DD831FF0128F3D0C821024800F0B1F8EEE740
S31508000DE870BD00BFBC5E000870B506460D461F4BB1
S31508000DF8D3F8C00201F038FD1D4B1C789CB91D4874
S31508000E08FFF754FF012801D0204670BD194B1B78FF
S31508000E18013BDBB23E2BF7D80122154B1A7000228C
S31508000E28154B1A70F0E7144B1B7801331148184410
S31508000E38FFF73CFF0446012801D00024E4E70E4BDF
S31508000E481A780132D2B21A700A4B1B789A4201D024
S31508000E580024D9E709493046FFF74EFB0022044B20
S31508000E681A70054B1B782B70CEE700BFD00A0020F6
S31508000E78D40D0020940D0020D50D0020950D0020D6
S31508000E8830B583B0144B1878FFF71AFF08B3054630
S31508000E98402800D94025002405E09DF807200F4B77
S31508000EA81A550134E4B2A5420DD90DF107010A4BCA
S31508000EB81878FFF7C9FE0128EFD04FF4A47108483F
S31508000EC800F03EF8E9E7ABB2044A8121054804F088
S31508000ED858FE03B030BD00BF480A0020D4090020D8
S31508000EE8BC5E0008D00A002070B5044604F01CFD54
S31508000EF8064621460F4804F0F2FD85B2002401E0B3
S31508000F080134A4B2AC420CD2315D0B4B1878FFF70A
S31508000F1861FE0128F4D04FF4B571084800F010F8BE
S31508000F28EEE704F001FD402302460121014804F0DA
S31508000F3830FE70BDD00A00208C0A0020BC5E00086E
S31508000F4808B500F007F9FCE708B500F0F7F8012836
S31508000F5803D00B4B1B78012B00D008BDFFF7FCFD0F
S31508000F68084B1B68084A1268134403F5FA73984233
S31508000F78F3D30022024B1A70FFF79EFAEDE700BF7B
S31508000F88DC0D0020D80D0020E00D0020014B18606C
S31508000F98704700BFD80D0020014B1868704700BF7E
S31508000FA8D80D002008B5054B1B78012B00D008BDC5
S31508000FB8FFF7D2FD024B1860F9E700BFDC0D0020E9
S31508000FC8E00D002008B50122034B1A70FFF7EAFF67
S31508000FD8FFF7BAFF08BD00BFDC0D002008B5FFF70C
S31508000FE867FA00F0B3F8FFF795FDFFF7B3FC00F0D2
S31508000FF80DF8FFF7E7FF08BD08B500F0ABF8FFF7EF
S315080010089DFD00F017F8FFF79FFF08BD10B500F023
S315080010180FFAFFF797F9064C01232370FFF7E6FC4A
S3150800102800232370FFF760FE0223237010BD00BF5C
S315080010380000002000B583B00DF107011848FFF736
S315080010480FFA012810D00DF107011548FFF706FD1C
S31508001058012812D00DF107011148FFF7C5FE01282E
S3150800106814D003B05DF804FB01220E4B1A709DF8E4
S3150800107807100B4800F0FCF9E5E70022094B1A703F
S315080010889DF80710064800F0F3F9E3E70222054B36
S315080010981A709DF80710024800F0EAF9E1E700BF60
S315080010A8E40D00200000002008B5FFF763FE08BD20
S315080010B838B504460D460E4B1B78012B09D00C4B48
S315080010C81B7853B10A4B1B78022B0BD000F0C8F9D2
S315080010D838BDC9B2FFF792F9F1E7E9B22046FFF73A
S315080010E8A1FCEFE7E9B22046FFF754FEEEE700BF9A
S315080010F800000020074B1B78022B05D0032B05D0D0
S31508001108012B05D0402070473F20704700207047C4
S315080011180820704700000020074B1B78022B05D0D3
S31508001128032B05D0012B05D0402070473F20704778
S3150800113800207047082070470000002008B500F016
S3150800114885F9034600B10123184608BD08B500F01D
S3150800115813FA08BD08B500F014FA08BD0022014BB9
S315080011685A707047240E0020034BFE22DA70187155
S315080011780222A3F844207047240E002010B5054C17
S3150800118800232370FFF7EAFFFF23E3700123A4F87F
S31508001198443010BD240E0020064BFF22DA700022C8
S315080011A81A71597859719A71DA711A720622A3F85E
S315080011B844207047240E002008B50020FFF7D4FF06
S315080011C808BD0000074BFF22DA70074A9A64002216
S315080011D81A715A719A710722C3F807200822A3F8C8
S315080011E844207047240E0020E45E0008044BFF22C2
S315080011F8DA7042689A640122A3F84420704700BF4F
S31508001208240E002008B53120FFF7AEFF08BD000000
S3150800121838B5084CFF23E370002525716571FFF77B
S3150800122869FFA071E571257265720723A4F8443031
S3150800123838BD00BF240E002038B5FFF78FFF0E4CC7
S3150800124801252570FF23E37010232371002363719A
S31508001258FFF750FFA071FFF75FFFE071FFF75CFF2C
S31508001268C0F3072020726572A5720823A4F84430D3
S31508001278FFF770FB38BD00BF240E002038B50546B9
S315080012884478FFF737FF0138844210DC0A4C6A783D
S31508001298A16C201DFFF730F9FF23E3706A78A36C69
S315080012A81344A3646B780133A4F8443038BD22206C
S315080012B8FFF75AFF38BD00BF240E002038B504468C
S315080012C84578FFF717FF0138854211DC61680A4D32
S315080012D8A9646278281DFFF70FF9FF23EB70627877
S315080012E8AB6C1344AB6463780133A5F8443038BD56
S315080012F82220FFF739FF38BD240E0020F8B5054629
S315080013081746002406E015F8013B1C44E4B2FFF72B
S3150800131821FF31464E1E0029F5D13C600120F8BD53
S3150800132810B5084CFF23E370E21D4168A06CFFF76F
S31508001338E5FF207100236371A3710823A4F84430DC
S3150800134810BD00BF240E002038B505460D4B9C6C11
S31508001358FFF7D0FE6A1C411E2046FFF7FFFA60B168
S31508001368084CFF23E370FFF7C5FE0138A36C034456
S31508001378A3640123A4F8443038BD3120FFF7F4FEEE
S3150800138838BD00BF240E002038B504464578FFF757
S31508001398B1FE023885420EDC114BFF22DA700122B3
S315080013A8A3F84420617851B9FFF7E8FA90B93120D3
S315080013B8FFF7DAFE38BD2220FFF7D6FE38BDA21C95
S315080013C8074B986CFFF7CAFA28B16178044A936CF8
S315080013D80B44936438BD3120FFF7C6FE38BD00BFFD
S315080013E8240E002008B54168074B986CFFF7BAFA2F
S315080013F830B1054BFF22DA700122A3F8442008BD54
S315080014083120FFF7B1FE08BD240E002008B5FFF706
S3150800141853F8034BFF22DA700122A3F8442008BDCB
S31508001428240E002008B589B2FFF742FE08BD000061
S31508001438054B00221A709A6483F84320A3F84420BF
S315080014489A705A70704700BF240E0020034B1B7809
S315080014580BB1012070470020704700BF240E0020FA
S315080014680022024B83F84320704700BF240E002051
S3150800147808B50378FF2B04D0354A1278012A14D008
S3150800148808BDFFF7D9FE324B93F84330012B5AD0E3
S315080014982F4BB3F944100029F2DD1846012380F8CA
S315080014A843300330FFF7BEFFEAE7C93B352B46D87A
S315080014B8DFE803F03345454245453F363C3945455F
S315080014C845454545454545454545454545454545B6
S315080014D84545454545454545454545454545241EEE
S315080014E81B2145454527452A2D30FFF7C7FECAE77C
S315080014F8FFF7E4FEC7E7FFF779FEC4E7FFF710FF33
S31508001508C1E7FFF75FFEBEE7FFF756FEBBE7FFF743
S3150800151843FEB8E7FFF732FEB5E7FFF715FFB2E770
S31508001528FFF732FFAFE7FFF773FEACE7FFF75AFF9F
S31508001538A9E7FFF76BFFA6E7FFF764FEA3E72020F6
S31508001548FFF712FE9FE71020FFF70EFEA0E700BF81
S31508001558240E002008B5074B1B6913F4005F03D057
S3150800156801231BB1002008BD0023FAE700F03EF866
S31508001578012008BD0008025808B5642000F008F8DC
S3150800158808BD08B500F00AF808BD704770477047E7
S31508001598014B1880704700BF700E002008B5FFF78A
S315080015A8DBFA0E4B1B6898420FD30D4B1B786BB9A9
S315080015B801220B4B1A7080220A4B9A61FFF7CCFA64
S315080015C8094B1B881844054B186008BD0022044BB4
S315080015D81A704FF40002034B9A61EFE7740E002065
S315080015E8720E002000040258700E00204FF4000204
S315080015F8014B9A61704700BF0004025810B5164B94
S315080016086FF00042DA670024DC674FF0FF32C3F850
S315080016188020C3F88040C3F88420C3F88440C3F800
S315080016288820C3F88840C3F88C20C3F88C40C3F8D0
S315080016389020C3F89040C3F89420C3F89440C3F8A0
S315080016489820C3F89840C3F89C20C3F89C4004F037
S315080016587BF8204610BD00BF00440258104B1B7883
S315080016680BB90120704710B504464FF47A70B0FBE1
S31508001678F3F30C4A1068B0FBF3F000F09BF868B96E
S315080016880F2C01D9012010BD002221464FF0FF304A
S3150800169800F060F8044B1C60002010BD012010BD46
S315080016A801000020080000200400002010B50320CF
S315080016B800F03EF801F028FD0F498B69C3F30323B0
S315080016C80E4AD35C03F01F03D8408B6903F00F0357
S315080016D8D35C03F01F0320FA03F3094A1360094B86
S315080016E818600020FFF7BAFF10B10124204610BD84
S315080016F8044603F079FFF9E7004402583C5F0008FE
S315080017080C0000200800002038B50446FFF72CFA1C
S315080017180546B4F1FF3F02D0044B1B781C44FFF77B
S3150800172823FA401B8442FAD838BD00BF01000020BE
S315080017380649CB6823F4E0631B041B0C000200F47B
S31508001748E0600343024A1A43CA60704700ED00E0A6
S315080017580000FA0530B4144BDB68C3F30223C3F15F
S315080017680704042C28BF04241D1D062D13D9033B82
S31508001778012505FA04F4013C2140994005FA03F3CA
S31508001788013B13401943002807DB0901C9B2074B77
S31508001798195430BC70470023EAE700F00F00090126
S315080017A8C9B2034B1954F4E700ED00E000E400E081
S315080017B814ED00E00138B0F1807F0AD2064B586074
S315080017C8F021064A82F823100020986007221A603A
S315080017D870470120704700BF10E000E000ED00E008
S315080017E830B4436B0468D4F884106F4A114041EA50
S315080017F88301C4F884100468D4F8841021F47F019E
S31508001808856B41EA0541C4F88410816B0B4404686A
S31508001818D4F88810114041EA8301C4F8881004688E
S31508001828D4F8881021F4FE01C56B41EA0541C4F8CD
S315080018388810C16B03EB41030468D4F8A010114063
S3150800184841EA8301C4F8A0100468D4F8A01021F46A
S31508001858FE01056C41EA0541C4F8A010046C416C08
S3150800186801FB04340368D3F8B010114041EA840137
S31508001878C3F8B0100368D3F8B01021F4FE01856CDC
S3150800188841EA0541C3F8B010836CC16C01FB0344F7
S315080018980368D3F8AC10114041EA8401C3F8AC10C8
S315080018A8036D416D01FB03430468D4F8F010114039
S315080018B841EA8301C4F8F0100468D4F8F01021F45A
S315080018C87C11856D41EA0541C4F8F010816D03EB7A
S315080018D841030468D4F8C0100A4042EA8303C4F8EE
S315080018E8C0300268D2F8C03023F47C13C16D43EACD
S315080018F80143C2F8C0300268D2F8C03023F07C53DE
S31508001908016E43EA0163C2F8C030426B274B1344A1
S315080019189B00C366826B03EB82020267C16B02EB0C
S31508001928C1024267046C416C01FB04F102EB8102B7
S315080019388267846CC16C01FB04F102EB8102C26701
S31508001948046D416D01FB04F102EB8102C0F88020A9
S31508001958816D02EBC102C0F88420C46D856E05FB53
S3150800196804F402EB8402C0F88820016E01FB05F135
S3150800197802EB8102C0F890200D498A420DD9D0F8A9
S315080019889C3043F02003C0F89C30032380F8983035
S31508001998012007E0002243F8042BD0F89020934250
S315080019A8F8D3002030BC70470300FFFF002B001057
S315080019B8FCD30040F0B44C68E4B90E698C68264339
S315080019C80C6846EA84460D6ACC6944EA05648D695A
S315080019D82C434D692C43CD682C43D0F88470806E0F
S315080019E803FB00F307EB830547F823606C600835AB
S315080019F8002015E00C698E6826430C68264346F0D5
S31508001A088046E0E71418E678A3781B0443EA0663D9
S31508001A18647843EA0423145C234345F8043B0430FA
S31508001A28CB89034CE35C9842ECD3F0BC704700BF03
S31508001A38EC5E00087047000030B595B004464C22A5
S31508001A48A04901A804F062F9002C00F0388123683F
S31508001A589D4A934220D094F898300BB3226893692C
S31508001A6823F010039361FFF77FF8054623689A6900
S31508001A7812F0080F1AD0FFF777F8401B0A28F5D98D
S31508001A88D4F89C3043F00103C4F89C30032384F847
S31508001A989830012015B030BD03F580736360DAE726
S31508001AA884F899302046FFF7C5FFD7E79A6942F0C8
S31508001AB801029A61FFF758F8054623689A6912F0F1
S31508001AC8010F0FD1FFF750F8401B0A28F5D9D4F8AB
S31508001AD89C3043F00103C4F89C30032384F89830FB
S31508001AE80120D7E79A6942F002029A61237C012B02
S31508001AF840D02268936943F040039361637C012BC5
S31508001B083ED02268936923F480439361A37C012B12
S31508001B183CD02268936943F4805393612268936999
S31508001B2823F44073A1680B4393612268936923F0F1
S31508001B38A40393612268136923F010031361E36809
S31508001B48012B29D0002B2CD0022B00F09B80226871
S31508001B58936943F0800393612268136943F010037D
S31508001B681361E368032B1CD12268936943F02003A9
S31508001B78936116E02268936923F040039361BDE7F1
S31508001B882268936943F480439361BFE7226893699F
S31508001B9823F480539361C1E72268936943F00403E9
S31508001BA893612268A369591EE369013B1B0243EA4C
S31508001BB84163216A01390B436169013943EA0143E3
S31508001BC8D361A368B3F5407F62D0236E33B1226828
S31508001BD8D2F8C030616E0B43C2F8C030E36D226E8E
S31508001BE8D3420DD02168D1F8C83023F00703A26E76
S31508001BF814A800EB820252F84C2C1343C1F8C830DB
S31508001C08236C6BB12168D1F8BC3023F00703626CEA
S31508001C1814A800EB820252F84C2C1343C1F8BC30C6
S31508001C28A36C73B12168D1F8BC3023F07003E26C59
S31508001C3814A800EB820252F84C2C43EA0213C1F8A6
S31508001C48BC30236D73B12168D1F8BC3023F4E06346
S31508001C58626D14A800EB820252F84C2C43EA022360
S31508001C68C1F8BC302268184B9A4222D00023C4F81F
S31508001C789430C4F89C30012384F898302046FFF73E
S31508001C88AFFD07E72268936943F02003936188E765
S31508001C982168A36A013BE26A013A43EA0223226BF6
S31508001CA8013A43EA0213626A013A43EA0243CB60FD
S31508001CB88BE76268936823F003039360D6E70120ED
S31508001CC8E8E600BF445D000800A0004090F8983098
S31508001CD8013BDBB2012B07D9D0F89C3043F002034D
S31508001CE8C0F89C3001207047CB680A68D2B9072B20
S31508001CF80ED08A68DB0643EA82730A6943EA024316
S31508001D084A691343C26E496842F821300020704771
S31508001D180A69CB691B0243EA02438A69134343F0FB
S31508001D286053EFE710B40A6942EA4372072B0ED0EC
S31508001D388C684B6943EA8473006F496800EBC104F1
S31508001D4840F83120636000205DF8044B70478B69C2
S31508001D58F2E790F89830DBB2012B07D0D0F89C3020
S31508001D6843F00403C0F89C3001207047022380F82A
S31508001D7898300268936923F0010393610023C0F839
S31508001D889C301846704770B590F89840013CE4B204
S31508001D98012C07D9D0F89C3043F00203C0F89C30D0
S31508001DA8012070BD93FAA3F5B5FA85F50668D6F845
S31508001DB8C040C4F30544A5420BD2D6F8CC4023420A
S31508001DC80FD0D0F89C3043F04003C0F89C3001206F
S31508001DD870BDD0F89C3043F02003C0F89C30012031
S31508001DE870BD93FAA3F3B3FA83F3FFF7E3FD002074
S31508001DF870BD90F89830DBB2022B07D0D0F89C302B
S31508001E0843F00803C0F89C30012070470368C3F8FC
S31508001E18D010002070470000F0B590F89840E4B25A
S31508001E28022C07D0D0F89C3043F00803C0F89C3041
S31508001E380120F0BD402937D041295BD0046DA14265
S31508001E487ED2C46F456D05FB01F504EB85044FF09A
S31508001E58000E256805F080455560002D78D125685F
S31508001E68C5F38A451560256805F000559560256807
S31508001E7805F000451561A588D561656805F47025DE
S31508001E88D560656805F480155561656805F400151B
S31508001E989561E57905F07F0515626568ED0F556268
S31508001EA804F1080500245BE00468D4F8A05015F48A
S31508001EB8FE0F0FD0D4F8A45015F07F0F12D0D4F81F
S31508001EC8A440C4F3052E446F456C05FB0EF504EBD8
S31508001ED88504BEE7D0F89C3043F02003C0F89C3050
S31508001EE80120F0BDD0F89C3043F48073C0F89C30CC
S31508001EF80120F0BD0468D4F8B05015F4FE0F0FD0D1
S31508001F08D4F8B45015F07F0F12D0D4F8B440C4F3FF
S31508001F18052E846FC56C05FB0EF504EB850498E75A
S31508001F28D0F89C3043F02003C0F89C300120F0BD5F
S31508001F38D0F89C3043F48073C0F89C300120F0BD7B
S31508001F48D0F89C3043F02003C0F89C300120F0BD3F
S31508001F58256825F06045156085E72E5D1E55013410
S31508001F68D689134FBE5DB442F7D340290BD0412911
S31508001F780ED01F2911D80268012303FA01F1C2F805
S31508001F8898100020F0BD0368C3F8A8E00020F0BD4B
S31508001F980368C3F8B8E00020F0BD026801F01F0125
S31508001FA8012303FA01F1C2F89C100020F0BD00BF16
S31508001FB8EC5E00080368D3F89820D3F89C001F291C
S31508001FC803D8CA4012F0010F17D01F2905D901F006
S31508001FD81F02D04010F0010F11D01F2907D901F0B0
S31508001FE81F01012000FA01F1C3F89C10704701206F
S31508001FF800FA01F1C3F898107047002070470020CE
S3150800200870470368D3F8CC300B4201D001207047DB
S3150800201800207047144BDB6813F0010F09D0124BE8
S31508002028124A5A6002F188325A60DB6813F0010FC7
S3150800203816D10D4BD3F80C3113F0010F12D00A4BF9
S315080020480A4AC3F8042102F18832C3F80421D3F8EE
S315080020580C3113F0010F01D1002070470120704799
S315080020680120704700207047002000522301674569
S315080020780D4BDA6842F00102DA60DB6813F0010FEB
S315080020880FD0094BD3F80C2142F00102C3F80C21F2
S31508002098D3F80C3113F0010F01D000207047012046
S315080020A870470120704700BF00200052F8B5054662
S315080020B80E46FEF759FD0746012E09D0374C14E09F
S315080020C8FEF752FDC01B854261D375B90320F8BDDA
S315080020D804240AE0324B1B6934EA03030CBF0123C4
S315080020E8002383B1B5F1FF3FEAD134F00403F1D0F8
S315080020F82B4BD3F8103124EA030333F000430CBF03
S3150800210801230023EDE7012E1AD0254BD3F8103109
S3150800211823F0684323F480135B0C5B0443F0004305
S3150800212833F0024219D01F498A691A438A61002B7B
S315080021380FDA23F000431A4AC2F814310120F8BD11
S31508002148174B1B6923F0684323F480135B0C5B0465
S31508002158E6E7134A53610120F8BD012E0CD0104B4F
S31508002168D3F8103113F4803F15D04FF480320C4B56
S31508002178C3F814210020F8BD094B1B6913F4803FE6
S3150800218807D04FF48032064B5A610020F8BD032069
S31508002198F8BD0020F8BD0020F8BD00BF0400008087
S315080021A800200052800E00202C4B1B7D012B51D09D
S315080021B870B50C4615460122284B1A7501F1784167
S315080021C8B1F5801F38D216460022244B9A6131464B
S315080021D84CF25030FFF76AFF034640BB012E2DD05C
S315080021E81F4AD2F80C3143F00203C2F80C31BFF388
S315080021F86F8FBFF34F8F082355F8042B44F8042B29
S31508002208013B13F0FF03F7D1BFF36F8FBFF34F8F6F
S3150800221831464CF25030FFF749FF0346012E13D0DA
S315080022280F49D1F80C2122F00202C1F80C2100212D
S315080022380A4A1175184670BD0226C5E7084AD368C2
S3150800224843F00203D360D2E70549CA6822F00202BE
S31508002258CA60ECE702231846704700BF800E0020C4
S315080022680020005201F00303032B24D011F0010FBC
S315080022780BD01D4BDA6822F03002DA60DA680243BE
S31508002288DA60DA6842F08802DA6011F0020F11D0D3
S31508002298154BD3F80C2122F03002C3F80C21D3F8D9
S315080022A80C211043C3F80C01D3F80C2142F088021C
S315080022B8C3F80C2170470C4BDA6822F03002DA6052
S315080022C8D3F80C2122F03002C3F80C21DA6802434D
S315080022D8DA60D3F80C211043C3F80C019A6942F066
S315080022E810029A61704700BF0020005230B411F0FE
S315080022F8010F0BD0104CE36823F4E663E360E36848
S3150800230842EA00252B4343F08403E36011F0020FE9
S315080023180FD00949D1F80C3123F4E663C1F80C311A
S31508002328D1F80C3142EA00221A4342F08402C1F875
S315080023380C2130BC704700BF00200052F8B5484B46
S315080023481B7D012B00F089800F460446444B012269
S315080023581A7500229A61436813F0010F0ED10026F8
S31508002368636813F0020F13D1002E71D12368012B6D
S3150800237817D04FF0FF333B60A56848E001214CF2BF
S315080023885030FFF793FE06460028E9D00126E7E70E
S3150800239802214CF25030FFF789FE0028E4D00126C6
S315080023A8E2E761682069FFF75DFF636813F0010FCC
S315080023B812D1636813F0020F4AD002214CF250304A
S315080023C8FFF774FE00B10126264AD2F80C3123F02D
S315080023D80803C2F80C313BE001214CF25030FFF7F4
S315080023E865FE00B101261F4AD36823F00803D360A7
S315080023F8DFE701214CF25030FFF758FE0646194A26
S31508002408D168194B0B40D3600FE006BB0135E3686A
S31508002418A26813449D421BD2226961682846FFF7C1
S3150800242865FF636813F0010FE3D1636813F0020FC1
S31508002438EBD002214CF25030FFF738FE0646094A1F
S31508002448D2F80C11084B0B40C2F80C31DDE73D6099
S315080024580022034B1A753046F8BD0226FBE700BF73
S31508002468800E002000200052FBF8FFFF2DE9F047F8
S3150800247882B0D0F80080CA00521A930003445A6DF5
S315080024881B6D9A4255D8C1469B1AC1EBC104A200D6
S315080024980244526C934200D81A460C46074602F183
S315080024A8030A4FEA9A0A15E006F1030A4FEA9A0A56
S315080024B8E3001B1B9D003D44A96C3B7C0093B3B20B
S315080024C8E2B2404601F0FEFFAB6C3344AB646B6D79
S315080024D81E446E6509EB441303F510639B699BB2AA
S315080024E89A4512D8E3001B1B9A003A44516D136D9E
S315080024F899420AD24BB15B1AC4EBC4018A003A4422
S31508002508566CB342D0D81E46CEE7E3001B1B98008C
S3150800251807443A6D7B6D9A420FD804F00F040123DD
S31508002528A340D8F8344824EA0304C8F834480020F5
S3150800253800E0012002B0BDE8F0870020FAE77047FE
S31508002548F0B58BB0002800F091800446056890F82D
S31508002558BD3323B3032384F8BD33EB6B13F4807FB1
S3150800256801D100232361206801F070FD254655F83E
S31508002578107B6E460FCD0FC60FCD0FC695E8030024
S3150800258886E80300231D0ECB384601F09DFC58B19A
S31508002598022384F8BD33012528460BB0F0BD80F820
S315080025A8BC33FFF7CCFFD5E70021206801F054FDBE
S315080025B8002315E0D900C81A82002244012082F8AF
S315080025C83D0082F83C30A2F84230002082F83F00ED
S315080025D850649064CA1A9100214408650133DBB235
S315080025E86568AB42E6D3002315E0D800C11A8A000D
S315080025F82244002182F8FD1182F8FC3182F8FF1185
S31508002608C2F80412C2F80812C21A90002044C0F888
S3150800261810120133DBB29D42E7D8254655F8107BE0
S315080026286E460FCD0FC60FCD0FC695E8030086E890
S315080026380300231D0ECB384601F054FD054660B944
S31508002648002384F83830012384F8BD33636A012BE4
S3150800265808D0206802F005F99EE7022384F8BD33FE
S31508002668012599E7204600F031FDF2E7012593E7B1
S315080026787047026890F8BC33012B19D010B50123AE
S3150800268880F8BC33836A012B0AD00446006802F036
S31508002698DCF8206801F0D4FC002084F8BC0310BDDF
S315080026A88369012BF1D0936B43F480339363ECE78A
S315080026B80220704738B590F8BC33012B02D10225A1
S315080026C8284638BD0446012380F8BC33006801F063
S315080026D8BDFC206802F085F8054620B1002384F879
S315080026E8BC330125ECE7206802F0BBF8002384F820
S315080026F8BC33E5E768B110B50446032380F8BD3353
S31508002708FFF7D8FF2046FFF7B3FF002084F8BD037C
S3150800271810BD01207047000070B504460D460068D4
S31508002728066C00EB411303F5306399682269012AA0
S3150800273811D0374A964254D03DB9C5EBC502930025
S315080027482344D3F81032002B5CD0E9B2204603F0B4
S31508002758F7F8002070BD11F0080F09D02D4A9642E7
S31508002768F7D911F4004FF4D04FF400429A60F0E715
S3150800277811F0200F28D111F0280FEAD1254A9642E0
S3150800278802D911F4004F22D1E900491B8A002244D4
S31508002798D2F804121B69C3F31203C91AC2F8141231
S315080027A8D2F80412D2F808320B44C2F8083235B9FE
S315080027B8C5EBC50293002344D3F810325BB1E9B2DE
S315080027C8204603F0BDF8C4E720229A60C1E74FF413
S315080027D800429A60BDE704F57172012102F092F889
S315080027E8EDE711F4004F09D111F0200F01D020228E
S315080027F89A60E9B2204603F0A3F8AAE74FF4004224
S315080028089A60A6E704F57172002102F07BF89CE746
S315080028180A31544F0A30544F38B5044603681D6CBC
S3150800282803EB4111D1F8082B0E4B9D4207D901F548
S31508002838306112F4004F02D04FF400438B602046F3
S3150800284803F076F8074B9D4202D92369012B01D07C
S31508002858002038BD04F571720121206802F052F88B
S31508002868F6E700BF0A30544F2DE9F84F04460568C5
S31508002878284602F032F808B1BDE8F88F2F46064612
S31508002888206801F0FAFF0028F6D0206801F0F5FF65
S3150800289810F0020F04D02268536903F0020353614B
S315080028A8206801F0EAFF10F0100F15D02268936926
S315080028B823F010039361D5F8208008F00F09C8F3B0
S315080028C84343022B00F08580062B00F0A58022687A
S315080028D8936943F010039361206801F0CEFF10F462
S315080028E8002F40F0AD80206801F0C7FF10F4802F54
S315080028F840F0F180206801F0C0FF0028C0F25F812F
S31508002908206801F0BAFF10F4006F0AD0D5F8083825
S3150800291813F0010F40F06D812268536903F40063D0
S315080029285361206801F0A9FF10F0006F15D02268DE
S31508002938536903F00063536194F8F433002B40F0AD
S315080029485C81012184F8F41323685B6DC3F3830360
S31508002958C4F8F833204600F0CDFB206801F08DFF57
S3150800296810F4805F40F04D81206801F086FF10F46E
S31508002978005F40F0AB81206801F07FFF10F0080F78
S3150800298840F0BC81206801F078FF10F4801F40F001
S31508002998BE81206801F071FF10F4001F40F0C18164
S315080029A8206801F06AFF10F0804F40F0C481206863
S315080029B801F063FF10F0040F3FF45EAF23685D680B
S315080029C815F0040F40F0C08123685A6815435D6006
S315080029D852E747F6F07318EA030F3FF478AF4FEA61
S315080029E8C90BABEB09034FEA830AA2444FEA181846
S315080029F8C8F30A02DAF80812284601F083FEC8F373
S31508002A080A08DAF808324344CAF80832DAF81432F7
S31508002A184344CAF814325AE7082204F5717128465D
S31508002A2801F070FEC8F30A184FEAC903A3EB0901B7
S31508002A388A002244D2F814324344C2F8143246E7CC
S31508002A48206801F01EFF8046B14617E007EB4913D8
S31508002A580122C3F8082B49462046FFF75DFE1DE00C
S31508002A6807EB49130822C3F8082B49462046FFF7FF
S31508002A78D3FE16E009F101094FEA5808B8F1000F24
S31508002A883FF431AF18F0010FF4D05FFA89F12068E6
S31508002A9801F007FF824610F0010FD7D11AF0080F88
S31508002AA8DED11AF0100F04D007EB49131022C3F829
S31508002AB8082B1AF0200F04D007EB49132022C3F875
S31508002AC8082B1AF4005FD5D007EB49134FF40052C8
S31508002AD8C3F8082BCEE7206801F0DBFE8046B1462E
S31508002AE82AE05946204602F037FF1AF0080F04D0A4
S31508002AF807EB49130822C3F808291AF0100F04D05F
S31508002B0807EB49131022C3F808291AF0400F04D016
S31508002B1807EB49134022C3F808291AF0020F04D014
S31508002B2807EB49130222C3F808291AF0800F41D186
S31508002B3809F101094FEA5808B8F1000F3FF4DAAE6F
S31508002B4818F0010FF4D05FFA89FB5946206801F09E
S31508002B58B1FE824610F0010FC7D009F00F03012114
S31508002B6801FA03F2D7F8343823EA0203C7F83438E7
S31508002B7807EB4913C3F8081923698B42B1D14FEA01
S31508002B88C902A2EB090293002344596C9A6C0A44B9
S31508002B989A64B9F1000FA4D1C9EBC902930023447A
S31508002BA81B6D002B9DD104F571720121206801F077
S31508002BB8A9FE96E749462046FFF758FCB8E7D5F830
S31508002BC8043823F00103C5F8043894F8F433012BC4
S31508002BD808D0204602F006FF2268536903F000432E
S31508002BE853618DE6002184F8F413204600F082FA32
S31508002BF8F2E7204602F0DCFE8EE6204602F0D8FE12
S31508002C08ABE605F50068D8F8043023F00103C8F8E0
S31508002C1804301021206801F037FA20E007EB461344
S31508002C284FF67F31C3F80819D3F8002922F40012A1
S31508002C38C3F80029D3F8002942F00062C3F800292E
S31508002C48C3F8081BD3F8002B22F40012C3F8002B8C
S31508002C58D3F8002B42F00062C3F8002B01366368EC
S31508002C689E42DBD3D8F81C3043F00113C8F81C3051
S31508002C78236BEBB1D8F8843043F00B03C8F88430DB
S31508002C88D8F8443043F00B03C8F84430D5F8003870
S31508002C9823F4FE63C5F8003804F57172217C2068B0
S31508002CA801F030FE2268536903F4805353615BE6EA
S31508002CB8D8F8142042F22B031343C8F81430D8F86E
S31508002CC8103043F00B03C8F81030DFE7206801F02E
S31508002CD809FE206801F0CAFAE060256800F00CFBD6
S31508002CE8227B0146284601F035F9204602F046FEC1
S31508002CF82268536903F4005353613CE6204602F000
S31508002D0836FE2268536903F0080353613AE6002140
S31508002D18204602F076FE2268536903F4801353614D
S31508002D2837E60021204602F066FE2268536903F456
S31508002D380013536134E6204602F069FE2268536997
S31508002D4803F08043536132E6204602F06AFE3BE60A
S31508002D58026890F8BC33012B16D010B5012380F809
S31508002D68BC33836A012B07D00446006801F06DFD61
S31508002D78002084F8BC0310BD8369012BF4D0936B3B
S31508002D8843F480339363EFE70220704790F8BC3327
S31508002D98012B01D10220704710B50446012380F89B
S31508002DA8BC33006801F05DFD002084F8BC0310BD43
S31508002DB890F8BC33012B01D10220704710B50446A0
S31508002DC8012380F8BC3380F83810006801F02DFD1F
S31508002DD8002084F8BC0310BDF8B511F0800F1ED189
S31508002DE801F00F06F500AF1BBC00274604F5FC7476
S31508002DF8044404343E460644002586F8FD5101F08D
S31508002E080F012170A260E370627802B1E180022B9B
S31508002E1814D090F8BC33012B13D10220F8BD01F069
S31508002E280F06F500AF1BBC002746383404440434A3
S31508002E383E460644012586F83D50E0E700232371FF
S31508002E48E7E70546012380F8BC332146006801F008
S31508002E581DFA002085F8BC03F8BD38B511F0800FB7
S31508002E6817D101F00F04E200151BAB001D4603F548
S31508002E78FC73034404332C460444002284F8FD21D9
S31508002E8801F00F01197090F8BC23012A10D102200D
S31508002E9838BD01F00F04E200151BAB001D46383398
S31508002EA8034404332C460444012284F83D20E7E70A
S31508002EB80446012280F8BC231946006801F02EFA58
S31508002EC8002084F8BC0338BD70B501F00F05EE0084
S31508002ED8711B8C0004F5FC740444211D761BB40090
S31508002EE80444C4F80822C4F810320023C4F814327B
S31508002EF884F8FD3184F8FC510369012B06D065B1C5
S31508002F08DAB2006801F0F2FA002070BDC5EBC50612
S31508002F18B4000444C4F80C22F1E7DAB2006801F0F8
S31508002F2845FAF1E701F00F01C1EBC1018B0018441E
S31508002F38D0F81402704770B501F00F05EE00711B42
S31508002F488C0038340444211D761BB4000444A2645A
S31508002F58236500236365012384F83D3084F83C50D3
S31508002F680369012B06D05DB1DAB2006801F0BEFA32
S31508002F78002070BDC5EBC506B4000444E264F2E758
S31508002F88DAB2006801F012FAF2E738B501F00F056F
S31508002F9843689D4238D811F0800F15D1CA00541AD3
S31508002FA8A3001C4603F5FC73034404332246024473
S31508002FB8002182F8FD1101229A701D7090F8BC2331
S31508002FC8012A0DD1022038BDEA00511B8B0019468B
S31508002FD83833034404330144012281F83D20EAE7E3
S31508002FE80446012280F8BC231946006801F09EFBB6
S31508002FF81DB1002084F8BC0338BD04F57172217C24
S31508003008206801F07FFCF4E7012038BD01F00F03C2
S31508003018426893422FD810B511F0800F14D1DA0000
S31508003028D41AA1000C4601F5FC7101440431044484
S31508003038002284F8FD2100228A700B7090F8BC33B0
S31508003048012B0DD1022010BDDA00D41AA1000C46B6
S315080030583831014404310444012284F83D20EAE762
S315080030680446012380F8BC33006801F08CFB002075
S3150800307884F8BC0310BD0120704730B40468606A40
S3150800308829B10D46A36A00EB134000230CE040EA79
S315080030980240A06212E003F1400104EB810149688D
S315080030A800EB11400133DBB2691E8B42F3D340EAC9
S315080030B8024005F13F0104EB81014860002030BC5D
S315080030C87047036859620020704700000246036883
S315080030D80121C0F8FC13002082F8F4039A6942F02B
S315080030E800629A61596D024A0A435A65704700BFD9
S315080030F80300001070470000024AD36843F0807343
S31508003108D360704700480258734B1B6903F03803AD
S31508003118102B00F0DF80182B11D00BB16F487047C1
S315080031286D4B1B6813F0200F01D16D4870476A4B29
S315080031381868C0F3C1006A4B23FA00F0704710B448
S31508003148654A916A01F00301906AC0F30510D46ACA
S3150800315804F00104536BC3F3CC0303FB04F307EE33
S31508003168903AF8EE677A002800F09480012966D02C
S31508003178F9B1022900F0918007EE100AF8EE476ABD
S315080031889FED586A86EE267A534B1B6BC3F30803E2
S3150800319806EE903AF8EE666A9FED536A67EE867A07
S315080031A876EEA77AF7EE006A77EEA67A27EE277AFA
S315080031B861E0494B1B6813F0200F23D046490A687B
S315080031C8C2F3C102464BD34007EE103AF8EE476AF7
S315080031D807EE100AB8EE476A86EE867A0B6BC3F3D3
S315080031E8080306EE903AF8EE666A9FED3F6A67EEC0
S315080031F8867A76EEA77AF7EE006A77EEA67A27EE4B
S31508003208277A38E007EE100AF8EE476A9FED376A1C
S3150800321886EE267A304B1B6BC3F3080306EE903A04
S31508003228F8EE666A9FED306A67EE867A76EEA77AD2
S31508003238F7EE006A77EEA67A27EE277A1BE007EEFE
S31508003248100AF8EE476A9FED276A86EE267A224B19
S315080032581B6BC3F3080306EE903AF8EE666A9FED11
S31508003268226A67EE867A76EEA77AF7EE006A77EE2E
S31508003278A67A27EE277A184B1B6BC3F34623013326
S3150800328807EE903AF8EE677AC7EE276AFCEEE67A12
S3150800329817EE900A5DF8044B704707EE100AF8EE29
S315080032A8476A9FED136A86EE267A0B4B1B6BC3F3A8
S315080032B8080306EE903AF8EE666A9FED0B6A67EE23
S315080032C8867A76EEA77AF7EE006A77EEA67A27EE7A
S315080032D8277AD0E7074870470044025800093D0096
S315080032E80090D0030024744A000000390024744C66
S315080032F80024F44A00127A0008B5FFF705FF0B4ABE
S315080033089369C3F303230A49CB5C03F01F0320FA26
S3150800331803F3926902F00F02885C00F01F0023FA93
S3150800332800F0044A1060044A136008BD00440258B5
S315080033383C5F00080C000020080000206A4B9842F1
S3150800334822D06A4B98422FD0694B98423CD0694B99
S31508003358984249D0684B984256D0684B984263D0F1
S31508003368674B984270D0674B98427DD0664B984217
S3150800337800F08A80654B984200F09680644B984224
S3150800338800F0A2800120704703F58843D3F8882007
S3150800339842F00102C3F88820D3F8882022F00102F7
S315080033A8C3F888200020704703F58043D3F888209F
S315080033B842F00202C3F88820D3F8882022F00202D5
S315080033C8C3F888200020704703F57053D3F888207F
S315080033D842F00402C3F88820D3F8882022F00402B1
S315080033E8C3F888200020704703F56053D3F888206F
S315080033F842F00802C3F88820D3F8882022F0080289
S31508003408C3F888200020704703F55053D3F888205E
S3150800341842F01002C3F88820D3F8882022F0100258
S31508003428C3F888200020704703F54053D3F888204E
S3150800343842F02002C3F88820D3F8882022F0200218
S31508003448C3F888200020704703F53053D3F888203E
S3150800345842F04002C3F88820D3F8882022F04002B8
S31508003468C3F888200020704703F52053D3F888202E
S3150800347842F08002C3F88820D3F8882022F0800218
S31508003488C3F888200020704703F51053D3F888201E
S3150800349842F48072C3F88820D3F8882022F4807210
S315080034A8C3F888200020704703F50053D3F888200E
S315080034B842F40072C3F88820D3F8882022F40072F0
S315080034C8C3F888200020704703F5E053D3F888200E
S315080034D842F48062C3F88820D3F8882022F48062F0
S315080034E8C3F88820002070470000025800040258D4
S315080034F800080258000C0258001002580014025816
S3150800350800180258001C02580020025800240258C5
S3150800351800280258F0B40C6894FAA4F4B4FA84F4AF
S315080035282EE08E68826803FB03F505EB450722EA59
S31508003538070205FB06F52A4382600E68CD684268CD
S3150800354822EA060205FB06F52A43426024E0466A93
S315080035581B0A03FB03F707FB03F707FB03F3C3EB96
S31508003568031726EA07074E6903FB06F33B4343623C
S315080035784B680668324005FB03F3134303600134BE
S315080035880B6833FA04F227D00122A2401340F6D07A
S315080035984A68013A012AC4D90F69C66803FB03F5C4
S315080035A805EB4502D243164005FB07F73E43C660BE
S315080035B84E68022EDCD1FF2BC9D8066A05FB03F72D
S315080035C807FB03F3C3EB031726EA07074E6903FB52
S315080035D806F33B430362CBE70020F0BC70470000C4
S315080035E82A4A136843F001031360284B1B6813F033
S315080035F8040F1AD10023002BF7D0244B00221A6196
S315080036081968234A0A401A60204B1B6813F0007F82
S315080036180DD00123002BF7D11C4B1B6813F0006F44
S3150800362807D00123002BF7D107E00123E3E700239E
S31508003638F0E70023F6E7002333B1144B1B6813F0B1
S31508003648005FF8D00123F7E7104B00229A61DA6188
S315080036581A62104999621049D962104919635A635E
S315080036689963DA6319645A64196821F48021196020
S315080036781A66996E40F2FF720A439A66D3F8D02002
S3150800368842F48032C3F8D020704700BF004402587D
S3150800369845EDF6EA000202020000FF018002010178
S315080036A807EE900AF8EE676A07EE901AF8EE677A58
S315080036B886EEA77A07EE902AF8EE677A06EE903A2B
S315080036C8F8EE666A9FED096A66EE866A77EEA67A66
S315080036D827EE277ADDED007AF8EE677AC7EE276ACD
S315080036E8FCEEE67A17EE900A704700BF000000392C
S315080036F82DE9F04182B04E4B9B6A03F00303012B78
S3150800370870D0002B5ED0022B77D0002600230360EA
S3150800371843608360464B9D6AC5F305151A6BC2F369
S315080037280802541CDB6A13F0010F77D00123002B1B
S3150800373876D03F4B5F6BC7F3CC07002D3FD03C4B89
S31508003748DB6A13F4803F6DD0012380466BB1384B92
S315080037581B6BC3F34623013300933B46224629468F
S315080037683046FFF79DFFC8F80000314BDB6A13F4B3
S31508003778003F59D001236BB12D4B1B6BC3F306438E
S31508003788013300933B46224629463046FFF788FF11
S31508003798C8F80400264BDB6A13F4802F46D00123A9
S315080037A86BB1234B1B6BC3F30663013300933B468C
S315080037B8224629463046FFF773FFC8F8080002B0C4
S315080037C8BDE8F0811A4B1B6813F0040F08D00123D3
S315080037D8F3B1174B1B68C3F3C103164EDE4095E7D2
S315080037E80023F5E7124B1B6813F4807F03D00123E7
S315080037F883B900268AE70023FAE70D4B1B6813F4FA
S31508003808003F03D001233BB900267FE70023FAE7E8
S3150800381800267BE7084E79E7084E77E7002386E710
S3150800382800278AE7002390E70023A4E70023B7E7E1
S31508003838004402580090D00300093D0000127A009F
S315080038482DE9F04182B04E4B9B6A03F00303012B26
S3150800385870D0002B5ED0022B77D000260023036099
S3150800386843608360464B9D6AC5F305359A6BC2F378
S315080038780802541CDB6A13F0100F77D00123002BBB
S3150800388876D03F4BDF6BC7F3CC07002D3FD03C4BB8
S31508003898DB6A13F4002F6DD0012380466BB1384BD1
S315080038A89B6BC3F34623013300933B4622462946BE
S315080038B83046FFF7F5FEC8F80000314BDB6A13F40B
S315080038C8801F59D001236BB12D4B9B6BC3F306435D
S315080038D8013300933B46224629463046FFF7E0FE69
S315080038E8C8F80400264BDB6A13F4001F46D00123E8
S315080038F86BB1234B9B6BC3F30663013300933B46BB
S31508003908224629463046FFF7CBFEC8F8080002B01B
S31508003918BDE8F0811A4B1B6813F0040F08D0012381
S31508003928F3B1174B1B68C3F3C103164EDE4095E780
S315080039380023F5E7124B1B6813F4807F03D0012395
S3150800394883B900268AE70023FAE70D4B1B6813F4A8
S31508003958003F03D001233BB900267FE70023FAE797
S3150800396800267BE7084E79E7084E77E7002386E7BF
S3150800397800278AE7002390E70023A4E70023B7E790
S31508003988004402580090D00300093D0000127A004E
S315080039982DE9F04182B04F4B9B6A03F00303012BD4
S315080039A872D0002B60D0022B79D000260023036042
S315080039B843608360474B9D6AC5F305551A6CC2F385
S315080039C80802541CDB6A13F4807F79D00123002B84
S315080039D878D0404B5F6CC7F3CC07002D18BF002E74
S315080039E83FD03C4BDB6A13F4800F6DD00123804629
S315080039F86BB1384B1B6CC3F34623013300933B4624
S31508003A08224629463046FFF74BFEC8F80000314BD8
S31508003A18DB6A13F4000F59D001236BB12D4B1B6CCD
S31508003A28C3F30643013300933B46224629463046EC
S31508003A38FFF736FEC8F80400264BDB6A13F0807FCA
S31508003A4846D001236BB1234B1B6CC3F306630133C2
S31508003A5800933B46224629463046FFF721FEC8F81A
S31508003A68080002B0BDE8F0811A4B1B6813F0040F72
S31508003A7808D00123F3B1174B1B68C3F3C103164ECD
S31508003A88DE4093E70023F5E7124B1B6813F4807FA3
S31508003A9803D0012383B9002688E70023FAE70D4BEC
S31508003AA81B6813F4003F03D001233BB900267DE7C2
S31508003AB80023FAE7002679E7084E77E7084E75E700
S31508003AC8002384E7002788E7002390E70023A4E774
S31508003AD80023B7E7004402580090D00300093D00C8
S31508003AE800127A00154B1B6903F03803182B0ED8F9
S31508003AF8DFE803F00F0D0D0D0D0D0D0D210D0D0D44
S31508003B080D0D0D0D160D0D0D0D0D0D0D18000020C2
S31508003B1870470A4B1B68C3F3C1030948D840704766
S31508003B280848704700B585B001A8FFF7E1FD019878
S31508003B3805B05DF804FB0448704700BF0044025806
S31508003B480090D00300127A0000093D00044B9B69D7
S31508003B5803F00F03034AD35C03F01F03D8407047EA
S31508003B6800440258FC5E0008044BDB69C3F30213E1
S31508003B78034AD35C03F01F03D84070470044025831
S31508003B88FC5E0008044BDB69C3F30223034AD35CD3
S31508003B9803F01F03D840704700440258FC5E00082B
S31508003BA800B585B0C2B2574BD358020EC0F30421EC
S31508003BB88A401340CB4040EA0340534B984228D0EA
S31508003BC831D8A3F58133A3F58073984263D019D801
S31508003BD8A3F5803398424ED003F54073984231D105
S31508003BE8FFF780FF494B9B69C3F30323484AD35C15
S31508003BF803F01F03D840FFF7A9FFFFF7C3FF05B077
S31508003C085DF804FB434B984245D003F57D4398423B
S31508003C1818D13E4B1B6813F0005F4CD00123002BCC
S31508003C284BD10020EBE73C4B98424DD00CD93B4B87
S31508003C38984256D003F54073984252D0A3F580337C
S31508003C48984241D00020DAE7A3F58033984203D09A
S31508003C5803F540739842F5D12C4B1B6813F0040FF3
S31508003C6830D00123002B4AD0284B1B68C3F3C10365
S31508003C782B48D840C3E7FFF735FF244B9B69C3F3A6
S31508003C880323234AD35C03F01F03D840FFF75EFFDC
S31508003C98FFF76AFFB3E71D4B1B6813F0006F03D0E5
S31508003CA801231BB90020AAE70023FAE701A8FFF7B2
S31508003CB8C7FD0298A3E70023B1E701A8FFF768FE46
S31508003CC802989CE70023CDE7104B1B6813F4807F06
S31508003CD803D001231BB1134891E70023FAE7002014
S31508003CE88DE70A4B1B6F13F0020F04D0012323B18B
S31508003CF84FF4004083E70023F9E700207FE7002018
S31508003D087DE700BF4C4402580803020700440258DE
S31508003D18FC5E0008080301070800040708000507F1
S31508003D280090D00300093D0038B5036813F0010F69
S31508003D383CD00123002B40F08E800D4604460368CC
S31508003D48464A1A408B6809690B4369690B43E9694E
S31508003D580B4313430360EB68426822F4405213434B
S31508003D684360AB69826822F44072134383603C4B14
S31508003D7898421DD03B4B98421ED03B4B98421FD0C9
S31508003D883A4B984220D03A4B984221D0394B984220
S31508003D9822D0394B984223D0384B984224D0002059
S31508003DA800284ED06A681ABB01204BE00023C1E7F9
S31508003DB83348FFF7F5FEF3E73248FFF7F1FEEFE77A
S31508003DC83048FFF7EDFEEBE72E48FFF7E9FEE7E791
S31508003DD82C48FFF7E5FEE3E72948FFF7E1FEDFE7AA
S31508003DE82848FFF7DDFEDBE72648FFF7D9FED7E7C1
S31508003DF82B68E9690B2B2CD8B1F5004F0DD0DBB22F
S31508003E08214951F82330B0FBF3F303EB5203B3FB14
S31508003E18F2F39BB2E360002014E0DBB21A4951F8CA
S31508003E282330B0FBF3F0530803EB4000B0FBF2F382
S31508003E384FF6F0721A40C3F342031343E3600020B7
S31508003E4800E00120E26A22F00F022B881343E3629E
S31508003E5838BD0020F6E7012038BD00BFF369FFEF3B
S31508003E68001001400044004000480040004C004053
S31508003E78005000400014014000780040007C0040D3
S31508003E8808030007080000070C5F00080023013331
S31508003E980C4A934211D80269002AF8DA036943F0F2
S31508003EA80103036100230133064A934207D80269CE
S31508003EB812F0010FF7D1002070470320704703203E
S31508003EC8704700BF400D030084B010B5044603A828
S31508003ED880E80E00089B012B0DD0E36843F04003E9
S31508003EE8E3602046FFF7D2FF0C9B13BBA36B43F492
S31508003EF88033A36311E0A36B23F48033A363E268DA
S31508003F08134B1340E360E36823F44013E3600F9B05
S31508003F18012B09D02046FFF7B9FF069B012B0DD0C8
S31508003F28BDE8104004B07047E36843F48013E360C3
S31508003F38F0E7A36B23F48033A363EEE7A36843F0A3
S31508003F480603A360A36843F02003A360E8E700BF5D
S31508003F58BFFFBDFF022A0AD00921C26822F470529F
S31508003F68C260C36843EA8123C36000207047274BB1
S31508003F780B44274A934239D9264B0B44264A93427F
S31508003F8836D9264B0B44264A934233D9254B0B443C
S31508003F9802F5C332A03293422ED9234B0B44234A47
S31508003FA893422BD9224B0B4402F5922202F57872DA
S31508003FB8934225D91F4B0B4402F5C32202F52072FA
S31508003FC893421FD91C4B0B4402F5B71202F55872D7
S31508003FD8934219D9194B0B4402F5122202F5F862D5
S31508003FE8934201D90621B8E70721B6E70F21B4E7B6
S31508003FF80E21B2E70D21B0E70C21AEE70B21ACE79D
S315080040080A21AAE70921A8E70821A6E7405327FFB6
S31508004018FF340C00401E1BFF3F420F0000DC0BFF5D
S315080040287F4F1200808CF9FE60B6E5FE5FE3160046
S3150800403800D3CEFEC05BB3FE00CA91FEE05459FE1B
S31508004048836843F00103836000207047836823F080
S31508004058010383600020704708B5C36823F0C0438E
S31508004068C360012909D069B9C36843F08043C360AE
S315080040783220FDF749FB002008BDC36843F000530A
S31508004088C360F5E7012008BD890141F020010161F7
S3150800409800230133054A934205D8026912F0200F16
S315080040A8F7D1002070470320704700BF400D030072
S315080040B81023036100230133054A934205D8026990
S315080040C812F0100FF7D1002070470320704700BF81
S315080040D8400D0300D0F800381943C0F8001800202E
S315080040E87047000084B02DE9F041044607A880E827
S315080040F80E002546002306E003F1400204EB82027F
S315080041080021516001330E2BF6D9119BA3BBD4F8B5
S31508004118043843F00203C4F80438A36B23F40013E5
S31508004128A363236843F040032360236843F08003AE
S3150800413823600023C4F8003E04F50066D4F8003866
S31508004148C4F800380C9B012B1BD003212046FFF727
S31508004158C1FF10212046FFF797FF804608B14FF0A8
S3150800416801082046FFF7A4FF08B14FF0010800230D
S3150800417833617361F3611BE0A36B43F40013A36314
S31508004188D7E7099B23B900212046FFF7A3FFE0E7F5
S3150800419801212046FFF79EFFDBE7C3B94FF0006011
S315080041A8C2F8000900220A614FF67F328A60013395
S315080041B807998B4210D205EB431202F51061D2F823
S315080041C800090028E9DB0020C2F80009EAE74FF0F1
S315080041D89040C2F80009E5E700230AE0BBB14FF0B2
S315080041E89047C2F8007B002202614FF67F32826050
S315080041F801338B4210D205EB431202F53060D2F830
S31508004208007B002FEADB0027C2F8007BEBE74FF0BC
S315080042180067C2F8007BE6E7336923F480733361E5
S315080042280023A3616FF0804363610A9B1BB9A369E6
S3150800423843F01003A361A2690A4B1343A3610D9BBC
S315080042481BB1A36943F00803A361119B012B04D092
S315080042584046BDE8F04104B07047A269024B1343D3
S31508004268A361F5E700383C8004000040D0F8083818
S3150800427813F0060305D0062B18BF022B03D102201C
S315080042887047002070470F207047000070B40B78FD
S315080042984A78012A20D0D0F81C2803F00F060124F2
S315080042A8B44042EA0442C0F81C2800EB4310D0F890
S315080042B8003B13F4004F0CD1D0F8002B8B68C3F3DE
S315080042C80A03C97843EA81431343134A1A43C0F8D1
S315080042D8002B002070BC7047D0F81C4803F00F0666
S315080042E8B24092B22243C0F81C2800EB4310D0F81B
S315080042F8002912F4004FECD1D0F800498A68C2F3B5
S315080043080A02C97842EA814242EA83532343024AA7
S315080043181A43C0F80029DCE70080001070B40C784E
S315080043284B78012B1FD0D0F83C5804F00F06012211
S3150800433802FA06F625EA0645C0F83C58D0F81C588D
S31508004348097801F00F018A4025EA0242C0F81C28BC
S3150800435800EB4410D0F8002B124B1340C0F8003B72
S31508004368002070BC7047D0F83C6804F00F0203FAC6
S3150800437802F292B226EA0202C0F83C28D0F81C28B3
S31508004388097801F00F018B409BB222EA0303C0F8B3
S315080043981C3800EB4410D0F80029034B1340C0F82A
S315080043A80039DDE70078F3EF007833EC70B40B7862
S315080043B84C78012C24D000EB431000F530631D69B6
S315080043C83E4C2C401C611D693D4C2C401C614C69B7
S315080043D80CB18C684C611C6944F400241C611C6986
S315080043E88D68C5F312052C431C61012A61D0D0F8E3
S315080043F8003B43F00443C0F8003B002070BC7047FC
S315080044084C695CBB00EB4314D4F810692C4D354055
S31508004418C4F81059D4F8105945F40025C4F81059A9
S31508004428D4F81069254D3540C4F81059012A31D0F9
S3150800443800EB4313D3F8002942F00442C3F80029D5
S315080044484B69002BD9D0D0F83428097801F00F0425
S315080044580121A1400A43C0F83428CEE700EB4314EB
S3150800446804F510642669154D354025612669144DED
S31508004478354025614E698D68AE4200D94D6125697A
S3150800448845F40025256125694E69C6F312063543A4
S315080044982561CBE70A691AB100EB4311C1F814295B
S315080044A800EB4310D0F8002942F00442C0F800296E
S315080044B8A3E7CA68002A9AD05A6198E70000F8FF65
S315080044C8FFFF07E070B49DF80C4064B903339E08F3
S315080044D807E000EB023303F5805351F8045B1D60CF
S315080044E80134B442F5D3002070BC7047F0B583B0E8
S315080044F80C784B78012B29D000EB441404F530636B
S315080045081E697D4D35401D611E697C4D35401D610E
S315080045184D69002D40F0C1801D698E68C6F31206E4
S3150800452835431D611D6945F400251D61012A00F002
S31508004538C980CB78012B00F0CB80D4F8003B43F038
S315080045480443C4F8003B002003B0F0BD4B6973BBB5
S3150800455800EB4413D3F81069684D3540C3F8105971
S31508004568D3F8105945F40025C3F81059D3F810693B
S31508004578614D3540C3F81059012A4AD000EB441456
S31508004588D4F8003943F00443C4F80039CB78012B32
S3150800459868D04B69002BD6D0D0F834380A7802F0A0
S315080045A80F0101228A401343C0F83438CBE700EBE1
S315080045B84413D3F81069504D3540C3F81059D3F849
S315080045C810694E4D3540C3F81059D3F810694D692E
S315080045D88F683D44013DB5FBF7F5494F07EAC545E0
S315080045E83543C3F81059D3F810594E69C6F312065D
S315080045F83543C3F8105903F51063CD78012DBBD19F
S315080046081D6925F0C0451D611D6945F000551D61E8
S31508004618B2E70B691BB100EB4412C2F81439CB7820
S31508004628012B08D000EB4414D4F8003943F00443AE
S31508004638C4F8003987E7D0F8083813F4807F08D11A
S3150800464800EB4412D2F8003943F00053C2F8003997
S31508004658E8E700EB4412D2F8003943F08053C2F871
S315080046680039DFE7D0F8083813F4807F0ED1D4F87C
S31508004678003943F00053C4F8003914460B46C96894
S315080046881A789B8A0094FFF71DFF5CE7D4F800396F
S3150800469843F08053C4F80039EFE78E683544013D86
S315080046A8B5FBF6F51E69164F07EAC5473E431E6170
S315080046B81F698E68ADB206FB05F5C5F312053D43BD
S315080046C81D6133E7CA68002A3FF433AF5A6130E7F9
S315080046D8D0F8083813F4807F06D1D4F8003B43F0A5
S315080046E80053C4F8003B28E7D4F8003B43F080534E
S315080046F8C4F8003B21E700BF0000F8FFFFFF07E00A
S315080047080000F81F03329208002393420CD210B413
S3150800471800F58054246841F8044B01339342F7D3D3
S3150800472808465DF8044B7047084670470B784A7880
S31508004738012A14D000EB4310D0F8002B002A06DB18
S315080047482BB1D0F8003B23F08043C0F8003BD0F8E3
S31508004758003B43F40013C0F8003B0020704700EB09
S315080047684310D0F80029002A06DB2BB1D0F8003907
S3150800477823F08043C0F80039D0F8003943F4001311
S31508004788C0F80039E9E70B784A78012A0ED000EB19
S315080047984310D0F8003B23F40013C0F8003BCB784D
S315080047A8023BDBB2012B15D90020704700EB4310FA
S315080047B8D0F8003923F40013C0F80039CB78023B47
S315080047C8DBB2012BF0D8D0F8003943F08053C0F893
S315080047D80039E9E7D0F8003B43F08053C0F8003BBE
S315080047E8E2E738B505460446002208E004EB42131A
S315080047F84FF67F31C3F80819C3F8081B01320E2A89
S31508004808F4D90022C5F81028C5F81428C5F81C28B4
S315080048182846FFF74DFC034608B1184638BD10214F
S315080048282846FFF731FC0346F7E7D0F8003823F4A3
S31508004838FE63C0F80038D0F80038090101F4FE61B3
S315080048480B43C0F800380020704708B5D0F804387C
S3150800485823F00203C0F804380320FCF755FF0020AC
S3150800486808BD08B5D0F8043843F00203C0F8043880
S315080048780320FCF749FF002008BD426980691040FB
S315080048887047D0F8183800F50060C0691840000C61
S315080048987047D0F8183800F50060C069184080B22B
S315080048A8704700EB4111D1F8082B00F50060406904
S315080048B81040704710B4D0F81028D0F8343801F0F2
S315080048C80F04E340DB01DBB2134300EB4111D1F8D7
S315080048D8080918405DF8044B7047406900F0010064
S315080048E870470000D0F80029054B1340C0F8003976
S315080048F8D0F8043843F48073C0F8043800207047A9
S3150800490800F8FFFF10B4046C154B9C4203D9D0F885
S31508004918003B002B16DB0024C0F8104BD0F8104BD0
S3150800492844F40024C0F8104BD0F8104B44F018048F
S31508004938C0F8104BD0F8104B44F0C044C0F8104BE0
S31508004948012903D000205DF8044B7047C0F8142BE2
S31508004958D0F8003B43F08023C0F8003BF2E700BFDD
S315080049680A30544F014B1860704700BF08000020F2
S3150800497898B108B50346D0F8B40210B10020C3F8B8
S31508004988B40209B1C3F8B0121846012380F89C325C
S31508004998027001F051F8002008BD0220704710B5D2
S315080049A80446012380F89C32D0F8B4325B68017952
S315080049B89847204601F0B2F8204601F09FF80020F3
S315080049C810BD19B1C0F8B41200207047022070470C
S315080049D808B501F09BF8002008BD08B5D0F8B43230
S315080049E823B11B68984718B1022008BD022008BDE4
S315080049F8002008BD08B5D0F8B4325B68984700208F
S31508004A0808BD38B5044600F52A75284600F04EF95B
S31508004A180123C4F89432B4F8AE32C4F8983294F83C
S31508004A28A81201F01F03012B0ED03BB1022B10D0A0
S31508004A3801F08001204601F08CF803E0294620465B
S31508004A4800F001FB002038BD2946204600F02FFB60
S31508004A58F8E72946204600F05AFBF3E738B5044636
S31508004A68A9BB1046D4F89432032B03D0052B25D0BE
S31508004A78002038BDD4F86031D4F8642193420DD9A2
S31508004A889B1AC4F860319A4206D99AB2014620465A
S31508004A9800F07AFC002038BD92B2F7E7D4F8B432B1
S31508004AA81B691BB194F89C22032A04D0204600F0FF
S31508004AB873FC002038BD20469847F7E70025C4F858
S31508004AC894522946204601F044F8284638BD0A4635
S31508004AD8D0F8B4329B694BB190F89C12032901D0DF
S31508004AE8022038BD11469847002038BD022038BD37
S31508004AF810B50446002956D11046D4F89432022B2C
S31508004B0809D0002B18BF042B44D094F8A032012BE7
S31508004B1845D0002010BD236A626A93421BD8E16912
S31508004B28B1FBF2F302FB13132BB98A4203D8D4F864
S31508004B38983299421DD3D4F8B432DB681BB194F87D
S31508004B489C22032A23D08021204601F002F8204619
S31508004B5800F02DFCD9E79A1A226292B2014620463D
S31508004B6800F00AFC00231A461946204601F011F8F7
S31508004B78CBE700221146204600F0FEFB0021C4F8C8
S31508004B8898120B460A46204601F003F8BDE7204668
S31508004B989847D8E78021204600F0DBFFB5E70020D4
S31508004BA884F8A00210BD0A46D0F8B4325B694BB146
S31508004BB890F89C12032901D0022010BD1146984787
S31508004BC8002010BD022010BD70B5044640230022FF
S31508004BD8114600F0ABFF0125C4F858514026C4F821
S31508004BE86461334600228021204600F09FFFA561B4
S31508004BF8666284F89C520023C4F894326360C4F849
S31508004C08A432D4F8B8322BB1D4F8B4325B68002190
S31508004C1820469847002070BD01740020704790F818
S31508004C289C3280F89D32042380F89C320020704715
S31508004C3890F89C32042B01D00020704790F89D32DA
S31508004C4880F89C32F8E708B590F89C32032B01D017
S31508004C58002008BDD0F8B432DB69002BF8D0984795
S31508004C68F6E700207047002070470020704708B50F
S31508004C78012280F89C22D0F8B4225268017990471C
S31508004C88002008BD002302E00133DBB201300278B8
S31508004C98002AF9D11846704708B54B88012B00D069
S31508004CA808BDC0F8A43200F077FBF9E70B78037063
S31508004CB84B7843708B78CA7803EB022343800B79C9
S31508004CC84A7903EB022383808B79CA7903EB02239B
S31508004CD8C380704710B50446802100F03AFF0021CA
S31508004CE8204600F036FF10BD30B583B005460C46A1
S31508004CF80023ADF806304A88130A013B062B00F252
S31508004D08C280DFE803F0041A30C0C09EAE00D0F8AF
S31508004D18B0321B680DF10601007C9847002353B989
S31508004D28BDF806201AB1E388002B40F0B280E38864
S31508004D38002B00F0B88003B030BD037C4BB9D0F81F
S31508004D48B4329B6A0DF10600984702234370002384
S31508004D58E5E7D0F8B432DB6A0DF106009847022376
S31508004D6843700023DBE7D2B2052A64D8DFE802F0ED
S31508004D78031323334353D0F8B0325B682BB10DF1D4
S31508004D880601007C98470023C9E72146FFF7A2FFDA
S31508004D9801230020C3E7D0F8B0329B682BB10DF188
S31508004DA80601007C98470023B9E72146FFF792FFDA
S31508004DB801230020B3E7D0F8B032DB682BB10DF138
S31508004DC80601007C98470023A9E72146FFF782FFDA
S31508004DD801230020A3E7D0F8B0321B692BB10DF1E7
S31508004DE80601007C9847002399E72146FFF772FFDA
S31508004DF80123002093E7D0F8B0325B692BB10DF197
S31508004E080601007C9847002389E72146FFF762FFD9
S31508004E180123002083E7D0F8B0329B692BB10DF146
S31508004E280601007C9847002379E72146FFF752FFD9
S31508004E380123002073E72146FFF74CFF01230020D2
S31508004E486DE7037C3BB9D0F8B4325B6B0DF106000D
S31508004E589847002363E72146FFF73CFF0123002014
S31508004E685DE7037C4BB9D0F8B4321B6B0DF106002D
S31508004E78984707234370002351E72146FFF72AFF7F
S31508004E88012300204BE72146FFF724FF01230020D2
S31508004E9845E79A4228BF1A46ADF80620014628462D
S31508004EA800F05DFA43E7284600F076FA43E738B596
S31508004EB804468B88F3B9CB88E3B94B887F2B19D876
S31508004EC803F07F0590F89C32032B0CD080F89E528D
S31508004ED8294600F04EFE204600F05EFA35B1022358
S31508004EE884F89C3238BDFFF7F5FE38BD012384F8EF
S31508004EF89C3238BD2046FFF7EDFE38BD38B5044666
S31508004F080D468978284B197001290ED890F89C32D5
S31508004F18022B0ED0032B21D02946FFF7DBFE224BA6
S31508004F2819782046FFF766FD38BD2946FFF7D2FEF1
S31508004F3838BD81B14160032380F89C32FFF74DFDE7
S31508004F48022803D0204600F027FA38BD294620460D
S31508004F58FFF7C0FE38BD00F01FFA38BD89B14368AF
S31508004F6899421DD0D9B2FFF745FD0F4B19786160F4
S31508004F782046FFF732FD02280DD0204600F00CFA2D
S31508004F8838BD022380F89C324160FFF733FD20467E
S31508004F9800F002FA38BD29462046FFF79BFE38BDC1
S31508004FA800F0FAF938BD00BF780E002008B5CB889E
S31508004FB8012B0BD190F89C329BB1022B09D9032BF4
S31508004FC80FD10122011D00F0CAF908BDFFF782FEBC
S31508004FD808BD0146002341F8083F012200F0BFF941
S31508004FE808BDFFF777FE08BD08B590F89C32013B67
S31508004FF8022B12D8CB88022B0CD10123C360D0F818
S31508005008A4320BB10323C360022200F10C0100F09D
S31508005018A6F908BDFFF75EFE08BDFFF75BFE08BDEB
S3150800502808B590F89C32013B022B09D84B88012B0E
S3150800503800D008BD0023C0F8A43200F0ADF908BDB9
S31508005048FFF748FEF5E708B50B7803F06003202B51
S3150800505805D0402B03D043B1FFF73CFE03E0D0F858
S31508005068B4329B689847002008BD4B78092B1BD893
S31508005078DFE803F011171A141A08051A0E0BFFF7BA
S3150800508833FEF0E7FFF713FFEDE7FFF737FFEAE729
S31508005098FFF78CFFE7E7FFF7A7FFE4E7FFF7FCFD55
S315080050A8E1E7FFF7BDFFDEE7FFF714FEDBE738B5F4
S315080050B805460C460B7803F06003202B05D0402BD9
S315080050C803D013B1FFF706FE0BE095F89C32013BB7
S315080050D8022B17D82379012B05D921462846FFF72D
S315080050E8F9FD002038BDD5F8B4329B682146284614
S315080050F89847E388002BF4D10028F2D1284600F017
S315080051084BF9EEE721462846FFF7E4FDE9E738B507
S3150800511804468A880B7803F06003202B08D0D0B29F
S31508005128402B05D05BB12046FFF7D4FD002038BDDB
S31508005138D4F8B4329B6820469847002038BD202BFF
S3150800514812D04B78012B3AD0002B67D0032B40F0AE
S31508005158E38094F89C32022B0CD0032B1DD02046F2
S31508005168FFF7B8FD002038BDD4F8B4329B6820464E
S31508005178984738BD002818BF802809D00146204618
S3150800518800F0E7FC8021204600F0E3FC002038BD4B
S315080051982046FFF79FFD002038BD4B882BB900280D
S315080051A818BF802801D0CB8823B1204600F0F4F830
S315080051B8002038BD0146204600F0CBFCF5E794F8F8
S315080051C89C32022B06D0032B17D02046FFF782FD08
S315080051D8002038BD002818BF802809D00146204677
S315080051E800F0B7FC8021204600F0B3FC002038BD4B
S315080051F82046FFF76FFD002038BD4B88002B40F08E
S31508005208908010F07F0F04D1204600F0C5F80020E2
S3150800521838BD0146204600F0A4FCF5E794F89C3210
S31508005228022B06D0032B2BD02046FFF753FD002070
S3150800523838BD002818BF802813D112F0800F15D161
S3150800524800F07F0000EB8000830003F5A871214475
S31508005258043100250D600222204600F080F8284611
S3150800526838BD2046FFF736FD002038BD00F07F0020
S3150800527800EB8000830003F1100121440431E8E7BC
S3150800528852B2002A20DB00F00F0303EB83039D00CC
S315080052982544D5F858312BB3002A28DB00F07F02BD
S315080052A802EB8202930003F5A87525440435802885
S315080052B818BF002825D100232B600222294620463C
S315080052C800F04DF8002038BD00F00F0303EB830308
S315080052D89D002544AB69002BDED12046FFF7FAFC72
S315080052E8002038BD2046FFF7F5FC002038BD00F041
S315080052F87F0202EB8202930003F110052544043568
S31508005308D5E70146204600F0D3FB10B101232B60F0
S31508005318D3E700232B60D0E72046FFF7DBFC002005
S3150800532838BD002038BDC8B170B50D4616460446C6
S31508005338FFF7A8FC013040003080287003236B7003
S31508005348022307E05A1CD2B20134E9540233DBB20D
S315080053580021A95421780029F4D170BD704710B5E9
S3150800536813460222C0F89422C36103620A46002142
S3150800537800F007FC002010BD08B513460A460021B0
S3150800538800F0FFFB002008BD08B513460A460021B1
S3150800539800F0FFFB002008BD08B50423C0F89432C6
S315080053A800231A46194600F0ECFB002008BD08B58C
S315080053B80523C0F8943200231A46194600F0E9FB7B
S315080053C8002008BD184AD2F8883043F47003C2F89A
S315080053D88830164B1A6842F001021A6000221A61D0
S315080053E818681349014019609A61DA611A629A6263
S315080053F8DA621A635A639A63DA631A645A6419682A
S3150800540821F4802119601A660A4B1A680A4B134058
S31508005418B3F1005F02D20122084B1A604FF000620E
S31508005428014B9A60704700BF00ED00E0004402583F
S315080054387FEDF6EA0010005C0000FFFF08810051C6
S3150800544808B55B4A136823F00F0343F00403136097
S31508005458136803F00F03042B03D067215548FBF79D
S315080054686FFD554AD36823F0070343F00203D36058
S31508005478936943F440439361504B1A6842F4802277
S315080054881A601A6842F480321A604C4B1B6813F487
S31508005498003F40F089800023002BF6D0474B9A6AD4
S315080054A822F0030242F002029A62DA6A42F4803271
S315080054B8DA62DA6A42F40032DA62DA6A22F00C024E
S315080054C842F00402DA62DA6A22F00202DA629A6AB8
S315080054D822F47C7242F040029A621A6B38491140EB
S315080054E840F2DF120A431A631A6B22F47E4242F428
S315080054F800721A631A6B22F4FE0242F498121A63AF
S315080055081A6B22F0FE4242F080721A631A6842F059
S3150800551880721A60294B1B6813F0007F46D1002356
S31508005528002BF7D0254B9A6922F00F0242F00802A1
S315080055389A611A6922F0070242F003021A619A6907
S3150800554822F470629A619A6922F00F0242F0080200
S315080055589A61DA6922F0700242F04002DA61DA6981
S3150800556822F4E06242F48062DA619A6922F07002F3
S3150800557842F040029A611A6A22F0700242F040022A
S315080055881A6210490A6822F007020A601A6D22F0A0
S3150800559840521A655A6D22F4401242F480125A652E
S315080055A80948FFF7DFF908BD012375E70123B7E7BF
S315080055B8002000524C5F0008004802580044025870
S315080055C800FEFFFF5444025800389C1C08B5FCF737
S315080055D86DF8FFF735FF08BD08B5FFF7F7FFFBF7C6
S315080055E8FDFCFBF709FDFCE72DE9F0418EB0514CAF
S315080055F8D4F8F43043F00203C4F8F430D4F8F4309D
S3150800560803F002030793079BD4F8E03043F001033D
S31508005618C4F8E030D4F8E03003F001030693069B9B
S31508005628D4F8E03043F00203C4F8E030D4F8E030A8
S3150800563803F002030593059BD4F8E03043F004030E
S31508005648C4F8E030D4F8E03003F004030493049B6C
S31508005658D4F8E03043F00803C4F8E030D4F8E03072
S3150800566803F008030393039BD4F8E83043F4802334
S31508005678C4F8E830D4F8E83003F480230293029B90
S31508005688D4F8EC3043F48073C4F8EC30D4F8EC3032
S3150800569803F480730193019B8023089301230993DC
S315080056A800250A950B950C95234F08A93846FDF74A
S315080056B831FF4FF40053089309950C9508A91F481C
S315080056C8FDF728FF4FF44078CDF820800226099682
S315080056D80A950B950C9507230D9308A91848FDF705
S315080056E819FFCDF8208009960A960B950C9509237B
S315080056F80D9308A93846FDF70DFF4FF4C0530893D4
S31508005708099603230A930B950C950A230D9308A962
S315080057180C48FDF7FFFED4F8D83043F00063C4F808
S31508005728D830D4F8D83003F000630093009B0EB045
S31508005738BDE8F081004402580004025800080258DF
S31508005748000C02580000025810B5FDF749FF214C15
S315080057584FF40003A3612048FDF7F0FD1F48FDF745
S31508005768EDFD2046FDF7EAFD1D48FDF7E7FD1D4B53
S31508005778D3F8D82022F00062C3F8D820D3F8EC2052
S3150800578822F48072C3F8EC20D3F8E82022F48022A9
S31508005798C3F8E820D3F8E02022F00802C3F8E0208E
S315080057A8D3F8E02022F00402C3F8E020D3F8E0207A
S315080057B822F00202C3F8E020D3F8E02022F0010222
S315080057C8C3F8E020D3F8F42022F00202C3F8F42044
S315080057D810BD00BF00040258000C02580008025801
S315080057E80000025800440258DFF834D0002103E0CC
S315080057F80C4B5B58435004310B480C4B42189A42E1
S31508005808F6D30B4A02E0002342F8043B094B9A42B6
S31508005818F9D3FFF7D7FD00F055FAFFF7DDFE704715
S3150800582800000220B45F000800000020C400002021
S31508005838C4000020E4140020FEE7000020230380AB
S3150800584800487047480000200A230380004870472C
S315080058586800002008B590F89C32032B01D0002078
S3150800586808BDFBF70DFBFAE708B5FBF709FB0020AF
S3150800587808BD08B50846FBF737FB002008BD000039
S3150800588808B50B7813F0600F06D14B780A2B14D09D
S315080058980B2B17D0062B01D0002008BD4B881B0AF6
S315080058A8212B04D00B491722FFF759FDF4E7CA88BC
S315080058B8172A28BF17220849F6E701220749FFF7DA
S315080058C84EFDE9E78B7813B9044A1360E4E7FFF756
S315080058D801FAE1E7510000205A0000207C0E00205A
S315080058E810B50446812100F02CF90121204600F064
S315080058F828F9002010BD000010B5044640230222EE
S31508005908812100F013F9402302220121204600F0E4
S315080059180DF94023034A0121204600F03AF90020F0
S3150800592810BD00BF9C0E0020004870479C0E002042
S3150800593808B500F57171D0F80404FFF762F808BDD8
S3150800594808B5C1EBC10293000344D3F80822D0F87E
S315080059580404FFF783F808BD08B5C1EBC102930034
S3150800596803449A6CD0F80404FFF7C2F808BD08B5D2
S31508005978D0F80404FFF767F908BD000010B5044617
S31508005988C3683BB1022B0FD091210848FBF7D8FA18
S31508005998012100E00021D4F80404FFF73DF9D4F802
S315080059A80404FFF711F910BD0121F4E7585F000850
S315080059B810B50446D0F80404FFF731F92268D2F87E
S315080059C8003E43F00103C2F8003E236A23B1044AA5
S315080059D8136943F006031361FBF7D8FD10BD00BF32
S315080059E800ED00E010B50446FBF7D1FDD4F8040431
S315080059F8FFF71EF910BD08B5D0F80404FFF733F908
S31508005A0808BD08B5D0F80404FFF72BF908BD10B58A
S31508005A1804460120FBF7B9FDD4F80404FFF725F975
S31508005A2810BD10B504460020FBF7AFFDD4F80404F2
S31508005A38FFF71DF910BD000003780BB10020704769
S31508005A4810B503461748C0F80434C3F8C002164B05
S31508005A580360092343600222C2600023036182614E
S31508005A680122C261036243628362C3620363FCF76D
S31508005A7867FD80B90B4C80212046FDF722FB4022A2
S31508005A8800212046FDF7F9FA802201212046FDF774
S31508005A98F4FA002010BD4FF493710448FBF750FA46
S31508005AA8E8E700BFDC0E002000000840585F000841
S31508005AB8D0F8C03211F0800F08D101F07F01C1EB90
S31508005AC8C1018A00134493F8FE01704701F07F016B
S31508005AD8C1EBC1018A00134493F83E00704708B524
S31508005AE8D0F8C002FDF71EFA08BD18B1022803D07F
S31508005AF802207047002070470120704708B5D0F883
S31508005B08C002FCF7F7FDFFF7F0FF08BD08B5D0F8A7
S31508005B18C002FCF7AEFDFFF7E8FF08BD08B5D0F8E8
S31508005B28C002FCF7C7FDFFF7E0FF08BD10B51C4625
S31508005B3813462246D0F8C002FDF74EF9FFF7D5FFFF
S31508005B4810BD08B5D0F8C002FDF787F9FFF7CDFFF5
S31508005B5808BD08B5D0F8C002FDF717FAFFF7C5FF64
S31508005B6808BD08B5D0F8C002FDF750FAFFF7BDFF23
S31508005B7808BD08B5D0F8C002FDF71AF9FFF7B5FF52
S31508005B8808BD08B5D0F8C002FDF7D5F9FFF7ADFF8F
S31508005B9808BD08B5D0F8C002FDF796F9FFF7A5FFC6
S31508005BA808BD000012230B800048704790000020AB
S31508005BB804230B8000487047A40000200023934262
S31508005BC816D230B40BE0373401F8134000015C00F4
S31508005BD8013400250D550133DBB2934206D2040F72
S31508005BE8092CF0D8303401F81340EFE730BC704779
S31508005BF87047000038B50A4B186804331C68043324
S31508005C081B68C01800D138BD064D0822A91CFFF725
S31508005C18D5FF042205F112012046FFF7CFFFF2E768
S31508005C2800E8F11FA800002008B51A230B80FFF723
S31508005C38E1FF014808BD00BFA800002008B50A46CC
S31508005C4828B105490548FFF76EFB034808BD024910
S31508005C580248FFF768FBF8E7E4120020985F000897
S31508005C6810B5044C0A4621460348FFF75CFB204654
S31508005C7810BD00BFE4120020885F000808B50A4670
S31508005C8828B105490548FFF74EFB034808BD0249F0
S31508005C980248FFF748FBF8E7E4120020685F0008A7
S31508005CA808B50A4628B105490548FFF73CFB0348E5
S31508005CB808BD02490248FFF736FBF8E7E412002058
S31508005CC8705F000870B50D4E0D4CA41BA410002576
S31508005CD8A54209D10B4E0C4C00F024F8A41BA410BD
S31508005CE80025A54205D170BD56F8253098470135D7
S31508005CF8EEE756F8253098470135F2E7AC5F000815
S31508005D08AC5F0008AC5F0008B05F000810B5431E1A
S31508005D180A44914200D110BD11F8014B03F8014F0E
S31508005D28F7E70000F8B500BFF8BC08BC9E46704700
S31108005D38F8B500BFF8BC08BC9E467047D2
S31508005D440000000000000000000000000000000041
S31508005D54000000000100000002000000030000002B
S31508005D640400000000000000050000000000000018
S31508005D74000000000000000006000000000000000B
S31508005D840000000000000000070000002E2E5C2E14
S31508005D942E5C2E2E5C2E2E5C536F757263655C41E9
S31508005DA4524D434D375F53544D333248375C636124
S31508005DB46E2E630005020602060307030803090399
S31508005DC409040A040B040C040C050D050E050F053D
S31508005DD40F0610061007100800000208000002004B
S31508005DE4010100000000040800000200020100008E
S31508005DF4000006080000020003010000000008086D
S31508005E04000002000401000000000A080000020065
S31508005E140501000000000C0800000200060100004D
S31508005E2400000E0800000200070100000000100828
S31508005E340000020000020000000012080000020030
S31508005E44010200000000140800000200020200001B
S31508005E5400001608000002000302000000001808EB
S31508005E64000002000402000000001A0800000200F4
S31508005E740502000000001C080000020006020000DB
S31508005E8400001E0800000200070200002E2E5C2EE9
S31508005E942E5C2E2E5C2E2E5C536F757263655C41E8
S31508005EA4524D434D375F53544D333248375C727302
S31508005EB43233322E630000002E2E5C2E2E5C2E2EDC
S31508005EC45C2E2E5C536F757263655C41524D434D6F
S31508005ED4375F53544D333248375C7573622E63000B
S31508005EE44F70656E424C5400000102030405060710
S31508005EF4080C1014182030400000000001020304A6
S31508005F040102030406070809010000000200000054
S31508005F140400000006000000080000000A00000053
S31508005F240C000000100000002000000040000000E3
S31508005F3480000000000100000000000001020304C4
S31508005F4401020304060708092E2E5C6D61696E2E8C
S31508005F54630000002E2E5C757362645F636F6E6661
S31508005F642E63000044656661756C740057696E5546
S31508005F7453422042756C6B20496E74657266616380
S31508005F84650000004F70656E424C54205573657267
S31508005F940000000057696E5553422042756C6B2009
S30D08005FA4446576696365000097
S30908005FACBD0200081C
S30908005FB0990200083C
S31508005FB404010000100000000090D0030090D003F4
S31508005FC401590008E958000889580008000000002B
S31508005FD400000000715800087B5800085D58000846
S31508005FE400000000000000000000000045580008FA
S31508005FF4000000005158000809022000010100C0F1
S31508006004320904000002FF0000000705810240006F
S31508006014FF070501024000FF0A06000200000040CF
S3150800602401000000AD5B0008B95B0008695C000864
S31508006034455C0008315C0008855C0008A95C00081A
S315080060441201000200000040501DAC60000201026B
S3150800605403010000040309041A03000000000000F9
S31508006064000000000000000000000000000000001E
S30908006074000000001A
S705080057F1AA
